:1000000093C0A5C0A4C0A3C0A2C0A1C0A0C09FC0EF
:100010009EC09DC09CC09BC09AC099C098C097C00C
:1000200096C095C094C06E616E00696E6600004017
:100030007A10F35A00A0724E18090010A5D4E800F7
:1000400000E87648170000E40B54020000CA9A3B0F
:10005000000000E1F5050000809698000000404295
:100060000F000000A0860100000010270000000023
:10007000E803000000006400000000000A00000027
:1000800000000100000000002C76D888DC674F08D3
:1000900023DFC1DFAE59E1B1B796E5E3E453C63AD9
:1000A000E651997696E8E6C28426EB898C9B62ED50
:1000B000407C6FFCEFBC9C9F40F2BAA56FA5F4900A
:1000C000055A2AF75C936B6CF9676DC11BFCE0E481
:1000D0000D47FEF520E6B500D0ED902E03009435D7
:1000E00077050080841E080000204E0A000000C82A
:1000F0000C333333330F986E12831141EF8D21147B
:10010000893BE65516CFFEE6DB18D1844B381BF74A
:100110007C1D901DA4BBE424203284725E228100E9
:10012000C9F124ECA1E53D2711241FBECFE5D4E0A1
:10013000DEBFCDBF10E0A0E6B0E0EEEDF0E102C022
:1001400005900D92A837B107D9F702D0C6C758CF8E
:10015000AF92BF92CF92DF92EF92FF920F931F93D5
:10016000DF93CF93CDB7DEB764970FB6F894DEBFB9
:100170000FBECDBFA7D021D17E010894E11CF11C98
:1001800090E6A92E90E0B92E8DE6C82E80E0D82EFC
:1001900085E090E064E670E027D12DB73EB72850A7
:1001A00030400FB6F8943EBF0FBE2DBF0DB71EB73F
:1001B0000F5F1F4FEDB7FEB7F282E182F801B38205
:1001C000A282A0E0B0E0BC01CD019FD12AE939E9CB
:1001D0004CE453E432D1F8016483758386839783BA
:1001E000FDD62DB73EB7285F3F4F0FB6F8943EBF00
:1001F0000FBE2DBFC701BBD080E062E0A3D084E07A
:1002000090E064E670E0F0D0EDB7FEB738970FB637
:10021000F894FEBF0FBEEDBF0DB71EB70F5F1F4FA7
:10022000F282E182F801D382C282A0E0B0E0BC0198
:10023000CD016BD12AE939E94CE453E4FED0F80151
:100240006483758386839783C9D62DB73EB7285FAD
:100250003F4F0FB6F8943EBF0FBE2DBFC70187D0EA
:1002600080E061E06FD094CF92B39F7092BB92B365
:10027000807F892B82BBC29A81E08A95F1F7C29870
:1002800008951F93182FC19AEFDF812F8295807FE9
:10029000EBDF8DE38A95F1F71F9108951F93182FD7
:1002A000C198E2DF812F8295807FDEDF88E38A9527
:1002B000F1F71F91089581E0F1DF80ED97E001975C
:1002C000F1F708950F931F9381B3806F81BB87B3BC
:1002D000866087BB82B38F7082BB88B3897F88BBFF
:1002E00088E99AE30197F1F780E3BEDF08E813E1BC
:1002F000C8010197F1F7C29A21E0822F8A95F1F7A0
:10030000C29888EE93E0FC013197F1F7C29A2A95E2
:10031000F1F7C2980197F1F780E2A6DFC8010197D3
:10032000F1F788E2BBDF8CE0B9DF86E0B7DFC3DF3F
:100330001F910F91089582E0B1DF80ED97E0019762
:10034000F1F70895623061F0633018F4613071F4B0
:1003500005C0633039F0643049F406C0805805C0E8
:10036000805403C0805701C0805398DF0895CF9315
:10037000DF93EC0102C0219684DF88818823D9F7BE
:10038000DF91CF9108950F931F93CF93DF938B014C
:10039000880F880F880F806481DFC0E0D0E0F8010B
:1003A000EC0FFD1F80816DDF2196C830D105B9F7B4
:1003B000DF91CF911F910F9108953F983E9A85E06C
:1003C00086B9379A369A3699FECF84B195B1089599
:1003D00097B18F71907E892B87B9369A3699FECF67
:1003E00024B135B1C9010895BF92CF92DF92EF9247
:1003F000FF920F931F93B82EC62EEE24FF24870181
:10040000DD2409C08B2DE4DFA0E0B0E0E80EF91E8A
:100410000A1F1B1FD394DC14A8F32C2D30E040E0FE
:1004200050E0C801B70167D4C9011F910F91FF9037
:10043000EF90DF90CF90BF9008950CD0BAC0B2D0AB
:1004400040F0A9D030F021F45F3F19F09BC051116A
:10045000E4C09EC0BFD098F39923C9F35523B1F3EC
:10046000951B550BBB27AA2762177307840738F023
:100470009F5F5F4F220F331F441FAA1FA9F333D082
:100480000E2E3AF0E0E830D091505040E695001C36
:10049000CAF729D0FE2F27D0660F771F881FBB1FF2
:1004A000261737074807AB07B0E809F0BB0B802DCC
:1004B000BF01FF2793585F4F2AF09E3F510568F018
:1004C00061C0ABC05F3FECF3983EDCF38695779557
:1004D0006795B795F7959F5FC9F7880F911D96951A
:1004E000879597F90895E1E0660F771F881FBB1F76
:1004F000621773078407BA0720F0621B730B840B23
:10050000BA0BEE1F88F7E0950895E89409C097FBB1
:100510003EF490958095709561957F4F8F4F9F4FDA
:100520009923A9F0F92F96E9BB279395F69587951E
:1005300077956795B795F111F8CFFAF4BB0F11F4E1
:1005400060FF1BC06F5F7F4F8F4F9F4F16C0882388
:1005500011F096E911C0772321F09EE8872F762FBE
:1005600005C0662371F096E8862F70E060E02AF0FF
:100570009A95660F771F881FDAF7880F96958795EB
:1005800097F9089597F99F6780E870E060E0089513
:100590009FEF80EC089500240A941616170618069B
:1005A0000906089500240A94121613061406050677
:1005B0000895092E0394000C11F4882352F0BB0F08
:1005C00040F4BF2B11F460FF04C06F5F7F4F8F4F6B
:1005D0009F4F089557FD9058440F551F59F05F3FA6
:1005E00071F04795880F97FB991F61F09F3F79F055
:1005F00087950895121613061406551FF2CF4695D7
:10060000F1DF08C0161617061806991FF1CF869558
:100610007105610508940895E894BB27662777273C
:10062000CB0197F90895A1E1B0E0E8E1F3E085C3DB
:100630003C017F876E876A01FC01178216828381E5
:1006400081FD03C06FEF7FEF52C39E012F5F3F4FCD
:10065000398B288BF3012381EE85FF8523FD85915E
:1006600023FF8191FF87EE87882309F43DC38532FC
:1006700051F4EE85FF8523FD859123FF8191FF874E
:10068000EE87853221F490E0B3017CD4E3CF982F3C
:1006900010E0882499241032B0F49B3269F09C3227
:1006A00028F4903251F0933271F40BC09D3239F03E
:1006B000903349F4116028C01260146025C018609E
:1006C00023C0106121C017FD2AC0892F80538A30B2
:1006D00078F416FF06C0FAE09F9E902C1124980E25
:1006E00013C03AE0839E802C1124880E10620CC047
:1006F0009E3221F416FDF8C2106406C09C3611F437
:10070000106802C0983659F4EE85FF8523FD959157
:1007100023FF9191FF87EE87992309F0BCCF892FA2
:100720008554833020F4812F8061905E07C0892F2B
:100730008556833008F08FC1812F8F7E86FD02C0E1
:1007400076E0972E6FE3F62EF822953619F4F0E452
:10075000FF2A07C0963619F420E8F22A02C0911049
:100760009A94F7FE0AC03BE3391518F45CE3B52E02
:1007700002C0B92CB39427E009C047E0491520F422
:10078000BB2447E0942EF7CF292DBB24C601049645
:100790009D878C87F6016081718182819381AE0192
:1007A0004F5F5F4F0B2D00D36C010981202E332446
:1007B00000FF04C003FD02C01DE209C0F1FE02C03B
:1007C0001BE205C0F2FC02C010E001C010E2C10152
:1007D0008C709070892BA1F1112311F483E001C07A
:1007E00084E0881510F0882409C0881AF3FC06C03C
:1007F00080E290E0B301C6D38A94D1F7112321F0AF
:10080000812F90E0B301BED323FE03C006E210E0C7
:100810000DC00AE210E00AC0E114F10409F08052B0
:1008200090E0B301AFD30F5F1F4F05C0EF2CFF2443
:10083000F0E1EF22FF24F8018491882369F708C1D1
:10084000F7FE12C0BC0C24FE04C08A81813309F477
:10085000BA941B141CF0BB24B3942DC0F8E0FB1514
:1008600050F538E0B32E27C0F6FC25C0892D90E066
:100870008C159D054CF02CEFC2162FEFD20624F0FC
:1008800030E8F32A01C09A94992049F0E2E0F0E0C0
:10089000EC0FFD1FE90DF11D80818033A1F3F7FE00
:1008A0000AC0B92CB394892D90E0C816D90614F06B
:1008B000992401C09C18F7FC03C025E030E009C072
:1008C0001C141D041CF021E030E003C096012F5FD2
:1008D0003F4F112311F02F5F3F4F992029F0892DB1
:1008E00090E00196280F391F882D90E028173907CE
:1008F00014F0882401C0821A4F2C5524C20189703B
:100900009070892B31F007C080E290E0B3013AD3B8
:100910008A948820C9F7112321F0812F90E0B30138
:1009200031D343FE06C007C080E390E0B3012AD371
:100930008A948820C9F7F7FE44C08601D7FE02C01A
:1009400000E010E076010894E11CF11CE01AF10AC5
:1009500041E050E04C0F5D1FE40EF51E26014B18E0
:100960005108892D90E0AA24BB24A81AB90A5FEF88
:100970000F3F150721F48EE290E0B30103D3C016B8
:10098000D10634F0401651061CF4F701808101C0F5
:1009900080E3015010400894E11CF11C0A151B056E
:1009A00024F090E0B301EED2E2CF0C151D0539F42E
:1009B0009A81963318F4953311F424FE81E390E084
:1009C00045C08A81813309F00F7E90E0B301DAD20D
:1009D000992091F08EE290E0B301D4D212E0E1E0F0
:1009E000F0E0EC0FFD1FE10FF11D1F5F808190E033
:1009F000B301C8D29A9499F744FC03C085E690E00D
:100A000002C085E490E0B301BDD2D7FC05C0C1149B
:100A1000D10441F404FF06C0D094C194D108D3940A
:100A20008DE201C08BE290E0B301ACD280E305C05F
:100A30008F5F26EF3FEFC20ED31E3AE0C316D104FC
:100A4000BCF790E0B3019ED2C601C096B3019AD222
:100A5000CC84DD8446C1933631F0933799F09335D9
:100A600009F055C022C0F601808189835E01089497
:100A7000A11CB11C22E030E0C20ED31E21E0E22E08
:100A8000F12C11C0F601A080B18016FD03C06FEFFC
:100A90007FEF02C0692D70E022E030E0C20ED31E6D
:100AA000C50165D27C011F7712C0F601A080B1801C
:100AB00016FD03C06FEF7FEF02C0692D70E022E0EA
:100AC00030E0C20ED31EC50147D27C01106813FF6F
:100AD00006C019C080E290E0B30154D28A94882DF8
:100AE00090E0E816F906B0F30EC0F50117FD859108
:100AF00017FF81915F0190E0B30144D281108A9485
:100B00000894E108F108E114F10479F7EAC0943699
:100B100011F0993681F517FF08C0F6012081318167
:100B20004281538184E090E00AC0F6018081918186
:100B30009C01442737FD4095542F82E090E0C80E79
:100B4000D91E9FE6F92EF12257FF09C05095409516
:100B5000309521953F4F4F4F5F4F90E8F92ACA01DA
:100B6000B901AE014F5F5F4F2AE030E058D2E82E66
:100B7000E889EE1A40C0953721F41F7E2AE030E064
:100B80001CC0197F9F3661F0903720F4983509F02A
:100B9000ABC00FC0903739F0983709F0A5C004C03A
:100BA00028E030E00AC0106114FD146020E130E05C
:100BB00004C014FD166020E132E017FF08C0F60102
:100BC000608171818281938144E050E008C0F60128
:100BD00080819181BC0180E090E042E050E0C40E51
:100BE000D51EAE014F5F5F4F1AD2E82E5889E51A25
:100BF0008FE7F82EF122F6FE0BC08EEFF822E914F3
:100C000038F4F4FE07C0F2FC05C09FEEF92202C0E2
:100C10001E2D01C0192DF4FE0DC0FE01EE0DF11DBB
:100C20008081803319F4E9EEFE2208C01F5FF2FED6
:100C300005C003C08F2D867809F01F5F0F2DF3FCD0
:100C400013C0F0FE0EC0181510F09E2C0AC09E2C8A
:100C5000980C911A182D05C080E290E0B30192D152
:100C60001F5F1815C8F304C0181510F4811A01C0CD
:100C7000882404FF0EC080E390E0B30183D102FF1B
:100C80001BC001FD03C088E790E00EC088E590E03E
:100C90000BC0802F867881F001FF02C08BE201C07B
:100CA00080E2F7FC8DE290E0B3016CD105C080E3F7
:100CB00090E0B30167D19A94E914C8F3EA94E1E0B3
:100CC000F0E0EC0FFD1FEE0DF11D808190E0B3010F
:100CD00059D1EE2099F705C080E290E0B30152D1DE
:100CE0008A948820C9F7B6CCF30166817781CB015D
:100CF0006196E2E13EC0A1E21A2EAA1BBB1BFD01D8
:100D00000DC0AA1FBB1FEE1FFF1FA217B307E407EA
:100D1000F50720F0A21BB30BE40BF50B661F771F42
:100D2000881F991F1A9469F7609570958095909522
:100D30009B01AC01BD01CF0108952F923F924F92CC
:100D40005F926F927F928F929F92AF92BF92CF925B
:100D5000DF92EF92FF920F931F93CF93DF93CDB764
:100D6000DEB7CA1BDB0B0FB6F894DEBF0FBECDBFDC
:100D700009942A88398848885F846E847D848C84AD
:100D80009B84AA84B984C884DF80EE80FD800C81B6
:100D90001B81AA81B981CE0FD11D0FB6F894DEBF99
:100DA0000FBECDBFED010895283008F027E03327AE
:100DB000DA01990F311D87FD91600096610571057B
:100DC00039F432602E5F3D9330E32A95E1F70895C0
:100DD0009F3F30F080387105610509F03C5F3C5F52
:100DE0003D93913008F08068911DDF93CF931F935E
:100DF0000F93FF92EF92192F987F9695E92F969572
:100E00009695E90FFF27E857FF4F99273327EE24E0
:100E1000FF24A701E70105900894079428F4360FF2
:100E2000E71EF81E491F511D660F771F881F991F67
:100E30000694A1F70590079428F4E70EF81E491FC1
:100E4000561FC11D770F881F991F661F0694A1F7B3
:100E50000590079428F4F80E491F561FC71FD11D8F
:100E6000880F991F661F771F0694A1F705900794B6
:100E700020F4490F561FC71FD81F990F661F771FF1
:100E8000881F0694A9F784911095177041F0D695A4
:100E9000C79557954795F794E7941A95C1F7EEE2F1
:100EA000F0E06894159015913591659195910590B4
:100EB0007FE27395E118F10A430B560BC90BD00979
:100EC000C0F7E10CF11E431F561FC91FD01D7EF451
:100ED000703311F48A95E6CFE894015030F0080F92
:100EE0000AF40027021708F4202F2395022F7A33E3
:100EF00028F079E37D932A95E9F710C07D932A9530
:100F000089F6069497956795379517951794E11884
:100F1000F10A430B560BC90BD00998F023957E912B
:100F200073957A3308F070E37C932013B8F77E91C1
:100F300070617D9330F0839571E37D9370E32A9522
:100F4000E1F71124EF90FF900F911F91CF91DF9166
:100F5000992787FD90950895FC0105906150704098
:100F60000110D8F7809590958E0F9F1F0895FC0172
:100F70006150704001900110D8F7809590958E0FC8
:100F80009F1F08950F931F93CF93DF938C01EB0165
:100F90008B8181FF1BC082FF0DC02E813F818C8120
:100FA0009D812817390764F4E881F9810193F98359
:100FB000E88306C0E885F985802F0995892B31F4EF
:100FC0008E819F8101969F838E8302C00FEF1FEF5A
:100FD000C801DF91CF911F910F910895AEE0B0E06D
:100FE000E3EFF7E0B8CE0D891E8986E08C831A8383
:100FF00009838FEF9FE79E838D839E01275E3F4F7E
:10100000CE0101966F89788DA9010DDB2F8138857E
:10101000020F131FF80110822E96E4E0B8CEFA01F9
:10102000AA27283051F1203181F1E8946F936E7F27
:101030006E5F7F4F8F4F9F4FAF4FB1E03ED0B4E018
:101040003CD0670F781F891F9A1FA11D680F791F59
:101050008A1F911DA11D6A0F711D811D911DA11D6A
:1010600020D009F468943F912AE0269F112430197A
:10107000305D3193DEF6CF010895462F4770405D15
:101080004193B3E00FD0C9F7F6CF462F4F70405DC4
:101090004A3318F0495D31FD4052419302D0A9F71F
:1010A000EACFB4E0A6959795879577956795BA9519
:1010B000C9F700976105710508959B01AC010A2EDF
:1010C00006945795479537952795BA95C9F7620FB6
:0E10D000731F841F951FA01D0895F894FFCF75
:1010DE0025382E336620416D706572650025382ED9
:0810EE00336620566F6C74009C
:00000001FF
